:03000000020100FA
:03000B00020B2EB7
:40010000D2D3D288758130C200757100C2A5C2A6C2A7C295D201D2A7D2951206F4120707120542120BD9120A8B75A800757B10C28CC28D5389F0758C00758A00C205D28CE3
:4001400075A90075A882300505C205120B67D2A230A246D2A130A14CD2A030A052D2A330A360D2A430A42C20A42C3001D975B003E5B05403F5F02323457185F071900A11EF
:4001800093B401053001BF4120B402053001B7611080B30208CB0208E4120539D2A230A276020146120539D2A130A171020146120539D2A030A063020146120539D2A202F0
:4001C00001463003121205FB12060712061312061F12064312075A20A4087800120886120785757C5690097712051BD2A330A3FB200302410112062B120637120643120757
:400200005A20A4087804120886120785757C5690097A12051B214602040202044B0204A2AA72BA01024138BA02024152BA0302416CBA0402418641A00566E566B43A0C754E
:400240006630E566757C16B1084152757C16B10861F70565E565B43A0C756530E565757C15B108416C757C15B10861F70564E564B43A0C756430E564757C13B108418675B6
:400280007C13B10861F70563E563B43A0C756330E563757C12B10841A0757C12B10861F70562E562B43A0C756230E562757C11B10841BA757C11B10861F70561E560B431A4
:4002C0000241C5400BE561B4350241CE4002D296E561B43A0C756130E561757C0FB10841EB757C0FB108120A8B61F70560120A8BE560B4330261025009E560757C0EB108A5
:40030000610E757C0E12082A12058F120A8B61F7AA72BA01026128BA02026142BA0302615CBA0402617661901566E566B42F0C756639E566757C16B1086142757C16B10868
:4003400061F71565E565B42F0C756539E565757C15B108615C757C15B10861F71564E564B42F0C756439E564757C13B1086176757C13B10861F71563E563B42F0C7563390D
:40038000E563757C12B1086190757C12B10861F71562E562B42F0C756239E562757C11B10861AA757C11B10861F71561E560B4310261B5500BE561B4350261C05002C29648
:4003C000E561B42F0C756139E561757C0FB10861DB757C0FB108120A8B61F71560120A8BE560B42F0B1207FC12058F120A8B61F5757C0EB10861F7120AAD12064312075A18
:400400002146200320D203757C1E90099012051B757C59900A0212051B1205B31205E31205EF020146C203757C1E90099612051B757C599009F312051B12061312058F1288
:40044000061F12064312075A0201460572E572B401028172B40202817EB40302818AB404028196757C0090096A12051B757205020146757C0090094012051B020146757CEB
:400480000090093312051B020146757C0090092612051B020146757C0090095D12051B0201461572E5726029B4010281C8B4020281D7B4030281E3B4040281EF757C009029
:4004C000096A12051B020146757C0090094012051B757201020146757C0090093312051B020146757C0090092612051B020146757C0090095D12051B020146D2901205346F
:40050000C290120534D29022C0E0E57C4480B129D0E0D29200F5800091FB22E493A3B4000122B108057C02051BC29200F5800091FBD292227FFFDFFE2278A079FFD9FED8E0
:40054000FA227438120529740C120529740612052974011205297400120529120534120534757C0E9008FDB11B757C19900959B11B12085812064312075A12058F75720203
:40058000757C0090093312051B1208A0C29622757C0E7860E612050808057CA97CB91004057CA97CB91404057CA97CB91702A1B2A19422757C597860E612050808057CA9CF
:4005C0007CB95B04057CA97CB95F04057CA97CB96202A1D6A1B82278677969E7F61809B85FF9227867798FE6F71819B85FF922781F796FE6F71819B817F92278677917E60C
:40060000F71819B85FF922781F7987E6F71819B817F9227867798FE7F61819B85FF922781F796FE7F61819B817F92278677917E7F61819B85FF922781F7987E7F61819B827
:4006400017F922757300757400757500757600757700E51FC394306007F578757900D1C7E51EC394306007F578757905D1C7E51DC394306007F57875790AD1C7E51CC394A3
:40068000306007F57875790FD1C7E51BC394306008F5787579141206C7E51AC394306008F5787579191206C7E519C394306008F57875791E1206C7E518C394306008F57885
:4006C0007579231206C722AE78900A53E579AF79933573F5730FEF933574F5740FEF933575F5750FEF933576F5760FEF933577F577DED622755EF812071A755EB012071A8A
:40070000755EC012071A22755EF812073A755EB012073A755EC012073A227810C2A7D2A6E55E20E702C2A6D2A5C2A5E55F33F55FE55E33F55ED8E7D2A7227810C295D2A695
:40074000E55E20E702C2A6D2A5C2A5E55F33F55FE55E33F55ED8E7D29522755E3085745F12071A755E2185755F12071A755E3285765F12071A755E2385775F12071A755E14
:400780005012071A22755E3085745F12073A755E2185755F12073A755E3285765F12073A755E2385775F12073A755E5012073A22C0E0C41207BED0E0057C1207BE22540F90
:4007C0004430B43A0280024002240712050822757C40E5771207B0057C057CE5761207B0057C057CE5751207B0057C057CE5741207B0057C057CE5731207B02275603075E1
:400800006130756230756330756430756530756630751830751934751A35751B30751C30751D30751E30751F302275603275613975623975633975643975653975663975E6
:400840001830751937751A34751B39751C39751D39751E39751F3922756030756137756230756337756430756530756630751830751935751A32751B30751C37751D307549
:400880001E30751F3022900A7BE42888F093F57708E893F57608E893F57508E893F5742220A414757C249009D112051BC206780412088612078522757C249009A612051BD0
:4008C000D206780012088612078522300613757C249009D112051BC206780412088612078502016A200613757C249009A612051BD206780012088612078502016A30302E17
:400900003030302E303000496E707574206E6577206672657175656E63793A30302E3030302E303030005354455020312020204B487A0053544550203130302020487A002E
:4009400053544550203130202020487A0056464F2D420056464F2D41004B487A005354455020313020204B487A005354455020313030204B487A00545800202000524954D9
:400980000020202000202000312057003520570053504C495400202020202000414D20203820202053005353420050757420612031342C323030204D487A207369676E6118
:4009C0006C20617420616E74656E6E6120616E64004357200043572020332C3120460043572020302C3420460043572020302C322046002020202020202020202020202076
:400A0000200020202E2020202E202020204B487A000001020302000301010300020302010040C00080C0804000000102020404040808080000000000000810101010101064
:400A400010202000000000000020202020202020202020006B000000003104000000F1290000006EA30100004D621000000AD7A30000666666060000000040013A92A301EE
:400A80003554751CC4EF881CD4AA10E560C3943023232323FCE561C394302CFD900A2993F57A757C40120AEFED1207B02285661F85651E85641D85631C85621BE561C39459
:400AC00030B4050241CA40065000D20441D0C204C3E5612405300404D4C39410F51AC3E5602404300403C32401F51975183022C294C2917808E57A33F57A50196103D8F509
:400B0000712722D29700000000D29100000000C291000041FEC29700000000D29100000000C291000041FE0000D294000022D57B10757B10C0D0C0E0120B42D205D0E0D081
:400B4000D032C2937E00D2B6D2B720B60BC2B7C3330EBE08F3020B60C2B7D3330EBE08E8F57DD293C2B722E57D757C5979407895E6FAE57DB50A026185400A09E9B44E02C3
:400B800061850861707B408B7C74FF1205080BE9B50B02619750F08B7C74201205080BEBB44F0261A740F0E9944075F004A4F5F0900C0593757C52120508057C05F0E5F0B7
:400BC00093120508057C05F0E5F093120508057C05F0E5F093120508227895760208762308763008763D08764608764F08765A08766A0876800876B30876BF0876E60876F9
:400C0000F00876F02231202020312020203220202033202020342020203520202036202020372020203820202039202020392B3130392B3230392B3330392B3430392B34B4
:010C40003083
:00000001FF
